:0200000480007A
:100000006F000005732F2034930F80006308FF03F7
:10001000930F90006304FF03930FB0006300FF038E
:10002000130F000063040F0067000F00732F2034CC
:1000300063540F006F00400093E19153171F0000BD
:1000400023223FFC171F000023200FFC6FF01FFF2F
:100050009300000013010000930100001302000050
:100060009302000013030000930300001304000038
:100070009304000013050000930500001306000020
:100080009306000013070000930700001308000008
:10009000930800001309000093090000130A0000F0
:1000A000930A0000130B0000930B0000130C0000D8
:1000B000930C0000130D0000930D0000130E0000C0
:1000C000930E0000130F0000930F0000732540F102
:1000D0006310050097020000938202017390523072
:1000E000735044749702000093820201739052305F
:1000F00073500018970200009382420273905230AE
:100100009B021000939252039382F2FF7390023B82
:100110009302F0017390023A73504030970200004E
:1001200093824201739052307350203073503030BC
:100130009301000097020000938202ED7390523009
:10014000130510001315F501635C05000F00F00F97
:10015000930110009308D005130500007300000000
:1001600093020000638A020073905210B7B200003D
:100170009B8292107390223073500030372500001C
:1001800073200530735030009702000093824201C3
:1001900073901234732540F17300203093012000D6
:1001A00017250000130505E683160500130520003A
:1001B000537005D473101000530500E4631AD5166C
:1001C00093013000172500001305E5E383160500B1
:1001D0001305E0FF537005D473101000530500E4BD
:1001E0006318D51493014000172500001305C5E1DD
:1001F0008316050013052000537015D473101000EA
:10020000530500E46316D512930150001725000032
:100210001305A5DF831605001305E0FF537015D401
:1002200073101000530500E46314D51093016000AF
:1002300017250000130585DD831605001305200032
:10024000537025D473101000530500E46312D50ECB
:100250009301700017250000130565DB8316050068
:100260001305E0FF537025D473101000530500E40C
:100270006310D50C9301800017250000130545D9A4
:100280008316050013052000537035D47310100039
:10029000530500E4631ED508930190001725000064
:1002A000130525D7831605001305E0FF537035D4D9
:1002B00073101000530500E4631CD5069301A000E1
:1002C00017250000130505D5071005008710250028
:1002D0000711450083166500D3012040D3F1014486
:1002E000538501E4F3151000130600006312D504D2
:1002F0006390C5049301B00017250000130505D2D3
:1003000007100500871025000711450083166500BA
:10031000D3012042D3F11144538501E4F3151000B9
:10032000130600006316D5006394C5006310300205
:100330000F00F00F638001009391110093E1110011
:100340009308D00513850100730000000F00F00F23
:10035000930110009308D0051305000073000000FE
:10036000731000C00000000000000000000000004A
:0C03700000000000000000000000000081
:1010000000000000000000000000000000000000E0
:1010100000000000000000000000000000000000D0
:1010200000000000000000000000000000000000C0
:1010300000000000000000000000000000000000B0
:081040000000000000000000A8
:10200000004000C00040007C004000C00040007C58
:1020100000BE0000000000BE00BE0000000000BEC8
:040000058000000077
:00000001FF
